:0200000480007A
:100000006F00C0006F20C02B6F20802B930000007A
:10001000130100009301000013020000930200008E
:100020001303000093030000130400009304000076
:10003000130500009305000013060000930600005E
:100040001307000093070000130800009308000046
:100050001309000093090000130A0000930A00002E
:10006000130B0000930B0000130C0000930C000016
:10007000130D0000930D0000130E0000930E0000FE
:10008000130F0000930F00009702000093820201FB
:10009000739052307350447497020000938202F7B9
:1000A0007390523017E100001301C1E3F32240F1D5
:1000B0009392C2003301510073100134EF20D0132A
:1000C000173500001305C5946F20407383328510E7
:1000D000739012148330850003310501833185014B
:1000E000033205028332850203330503833385031C
:1000F00003340504833485048335850503360506FA
:1001000083368506033705078337850703380508D7
:10011000833885080339050983398509033A050AB7
:10012000833A850A033B050B833B850B033C050C97
:10013000833C850C033D050D833D850D033E050E77
:10014000833E850E033F050F833F850F033505056D
:10015000730020107311011423341100233C31006B
:10016000233041022334510223386102233C7102BF
:1001700023308104233491042338A104233CB104A7
:100180002330C1062334D1062338E106233CF1068F
:10019000233001092334110923382109233C310973
:1001A0002330410B2334510B2338610B233C710B5B
:1001B0002330810D2334910D2338A10D233CB10D43
:1001C0002330C10F2334D10F2338E10F233CF10F2B
:1001D000F312011423385100F32200102330511080
:1001E000F322101423345110F32230142338511009
:1001F000F3222014233C5110130501006F20C03757
:1010000000000000000000000000000000000000E0
:1010100000000000000000000000000000000000D0
:1010200000000000000000000000000000000000C0
:1010300000000000000000000000000000000000B0
:081040000000000000000000A8
:10200000B367B500B3E7C70093F77700B306C50021
:10201000638407023386C50093070500637ED502FB
:1020200003C705009385150093871700A38FE7FE6C
:10203000E398C5FE67800000E37ED5FE93070500A8
:1020400003B70500938787009385850023BCE7FECF
:10205000E3E8D7FE6780000067800000130101FFFE
:10206000B367C500233081002334110093F7770054
:10207000130405003307C500638207026376E50099
:1020800093F5F50FEFF09FFD8330810013050400F9
:1020900003340100130101016780000093F5F50F7F
:1020A0009717000083B707E9B385F502E37EE5FCE7
:1020B000930705009387870023BCB7FEE3ECE7FE98
:1020C0008330810013050400033401001301010172
:1020D0006780000083470500638E070093070500B3
:1020E00003C7170093871700E31C07FE3385A7403B
:1020F000678000001305000067800000834705002B
:10210000938515001305150003C7F5FF638A0700C3
:10211000E386E7FE1B8507003B05E540678000007E
:10212000130500006FF05FFFB367B50093F777000A
:10213000639E0702137886FF330805016378050361
:10214000930705006F000001938787009385850042
:1021500063F8070183B6070003B70500E386E6FED0
:102160003385A7403306A640138507003386C50094
:102170006F00400103C705008347F5FF93851500F5
:10218000639AE70013051500E396C5FE13050000EA
:10219000678000003B85E7406780000093070500EB
:1021A00003C705009387170093851500A38FE7FEEB
:1021B000E31807FE6780000003470500930600024E
:1021C000930705006318D70003C71700938717000C
:1021D000E30CD7FE9306D0026300D7069306B00245
:1021E0006300D70483C607009305000063820604DA
:1021F0001305000093871700131725001B8606FDA3
:1022000083C607003307A700131717003305E6003E
:10221000E39206FE638005023305A040678000005C
:1022200083C617009305000093871700E39206FC0E
:10223000130500006780000083C617009305100097
:1022400093871700E39606FA130500006FF09FFED0
:1022500083470500638007049305101017F7FFFFFD
:10226000130747DA93950503033607001305150096
:10227000B3E6B700630A060097F7FFFF23B407DC55
:1022800083370700E39A07FE2330D7008347050012
:10229000E39C07FC6780000017F7FFFF130787D652
:1022A00083370700638A070097F7FFFF23BC07D82F
:1022B00083370700E39A07FE2330A7006F00000072
:1022C000130101FF1305903423341100EFF0DFFCFC
:1022D000130101FE1306810093077101130890009A
:1022E0006F008000930707009376F50013870600C0
:1022F000930500036374D800930570053B07B7008E
:102300002380E700135545001387F7FFE31CF6FC15
:1023100083478100230C010063820704130510101A
:102320009306060017F7FFFF1307C7CD1315050324
:10233000833507009386160033E6A700638A0500FD
:1023400097F7FFFF23B007D083370700E39A07FE14
:1023500083C706002330C700E39C07FC130101027A
:1023600067800000130101FB9307100037F7FFFFA0
:102370002322F1002334110423308104233C9102F1
:10238000233821032334310323304103233C5101FB
:1023900023340100B306E500B7E7030063F6F6183F
:1023A0009359C5009384096017490000130989C532
:1023B00093973400B307F90083B707003374E5003F
:1023C0006396071017870000130747C4033A0700F6
:1023D00063000A1883378A009786000083B686C296
:1023E0002330F700638CD712130641009305810058
:1023F00013050400833A0A00EF00C0606310051063
:1024000093D6CA009396A60093E6F60193973400FC
:10241000B307F90013E7060C23B0E70073000412BA
:1024200097370000938707BE93994900B387370118
:1024300003B707006318071203370A00B705040043
:1024400023B0E70003378A0023B4E700F3A50510A3
:10245000B707E0FFB307F4003716000013070400C6
:102460003386C70003B3070083B8870003B80701AA
:1024700003B5870123306700233417012338070190
:10248000233CA7009387070213070702E39CC7FCBE
:102490007390051093973400B304F90023B0D4006F
:1024A000730004120F100000833081040334010410
:1024B000833481030339010383398102033A010222
:1024C000833A8101130101056780000013F70704B7
:1024D0006302070413F70708631207061307F000E7
:1024E00093E70708639CE50493943400B3049900D0
:1024F00023B0F400730004126FF01FFB83360A0050
:102500008337810093D6C6009396A600B3E6F60003
:102510006FF0DFEF93E707046FF01FFD9787000070
:1025200023B207AE6FF05FEC17150000130505A18D
:10253000EFF01FD213053000EFF01FD61715000083
:10254000130545A4EFF0DFD013053000EFF0DFD422
:1025500017150000130585A7EFF09FCF1305300076
:10256000EFF09FD3171500001305C5A7EFF05FCE5E
:1025700013053000EFF05FD2130101F82338810614
:10258000233C11062334910623302107233C3105D7
:10259000233841052334510523306105233C710361
:1025A00023388103233491032330A103233CB10159
:1025B00013040500EF0080446312050E8335841177
:1025C000930780006380F510930720006380F50671
:1025D000938745FF130710006376F7009307F00019
:1025E000639CF51E03350411EFF0DFD713050400DB
:1025F00003340107833081078334810603390106E0
:1026000083398105033A0105833A8104033B0104C0
:10261000833B8103033C0103833C8102033D0102B0
:10262000833D8101130101086FD05FAA0337841035
:1026300093773700639E0706EF0780007310300022
:102640000327070083A707006300F7061305101090
:1026500093071004971600009386C69C17F7FFFF98
:102660001307479A13150503833507009386160051
:1026700033E6A700638A050097F7FFFF23B4079CA2
:1026800083370700E39A07FE83C706002330C7009D
:10269000E39C07FC13053000EFF01FC01305040096
:1026A000EFD0DFA26FF09FF113051000EFF0DFBE57
:1026B00017150000130505A1EFF09FB913053000B1
:1026C000EFF09FBD83270405B7140000973A000080
:1026D000938A4A932334F100174D0000130D8D9215
:1026E000B70C0400370CE0FF178A0000130A8A9128
:1026F000978B0000938B8B9137FB030093D7C4001B
:102700001399470033872A0103370700630C070832
:102710009387076093973700B307FD0083B90700DD
:1027200093F709046380070AF3AD0C103384840126
:10273000371600009305040013850400EFF0DF9EB8
:102740006304050493F909086380090AB7160000B9
:102750001387040093070400B386D40003380700EE
:1027600003358700833507010336870123B007014E
:1027700023B4A70023B8B70023BCC7001307070280
:1027800093870702E31CD7FCB3872A0173900D10CF
:1027900003370A0023B00700630007022334F70061
:1027A0002330FA00B7170000B384F400E39864F50F
:1027B00003358100EFF05FAE2330FA0023B0FB0059
:1027C0006FF05FFE171500001305C588EFF05FA8D6
:1027D00013053000EFF05FAC1715000013050591ED
:1027E000EFF01FA76FF01FEB171500001305058A08
:1027F000EFF01FA613053000EFF01FAAF32740F1FA
:10280000639A0718975700009387C77F130101ED5C
:1028100093D7C70023308112176800001308887E01
:10282000130405009397A700174500001305857D45
:10283000233411129356C5001357C80093E71700AD
:10284000973800009388087C1306F0FF233CF5FEC0
:102850009396A6001317A700B707002093E616006B
:102860001367170093D5C8001313F6039387F70C6B
:10287000233CF8FE23B0D8002330E500B3E7650021
:102880007390071873270018639EE7141356B60059
:102890009307F0019702000093824201F3925230B5
:1028A0007310063B7390073A739052301308F0BFD1
:1028B0001318580197E7FFFF9387078AB38707012B
:1028C00073905710F3270034B387070173900714F0
:1028D000B7B700009B87071073902730B7E7010058
:1028E0009B870760739007307350403017370000A4
:1028F000130747B09307083EB3060701B307F70075
:10290000B7080800177600002332D670173300008E
:10291000130343ED9776000023B6F66E9388F80311
:10292000930790021308080113D61700B386170106
:10293000B347F600B30507019396C6009397570077
:102940002330D7002334B70093F70702130707019A
:10295000B367F600E31AE3FC1306001293050000C8
:10296000130501009737000023BA07E6EFF00FEFD9
:10297000B70700803304F4001305010023348110ED
:10298000EFD0CFF48330811203340112130101130D
:102990006780000013071000B717FB063706080012
:1029A0009387A7A01306C6FF1315F7019316E70335
:1029B0006F00C0012F20070013D71700B3C7E7002F
:1029C0009397E703B3F7D700B3E7E70033F7C70000
:1029D00093F517003307A700E39E05FC03200700CB
:1029E0006FF09FFD1705000013054573EFF05F863C
:1029F00013053000EFF05F8A6780000013050000C8
:102A0000678000001305000067800000930120002C
:102A1000971000009380005F3701AA001B01A10AF4
:102A2000970700009387470123A0200003A7000019
:102A30006F00800013070100B703AA009B83A30A5D
:102A40006318774C93013000971000009380805BEF
:102A500037B100AA1B0101A0970700009387470127
:102A600023A2200003A740006F008000130701008D
:102A7000B7B300AA9B8303A0631C7748930140006F
:102A800097100000938000583711A00A1B0101AA7B
:102A9000970700009387470123A4200003A7800025
:102AA0006F00800013070100B713A00A9B8303AADD
:102AB0006310774693015000971000009380805474
:102AC00037A10AA01B01A1009707000093874701C7
:102AD00023A6200003A7C0006F0080001307010099
:102AE000B7A30AA09B83A3006314774293016000FD
:102AF000971000009380C0523701AA001B01A10A61
:102B0000970700009387470123AA20FE03A740FFF1
:102B10006F00800013070100B703AA009B83A30A7C
:102B20006318773E93017000971000009380404F28
:102B300037B100AA1B0101A0970700009387470146
:102B400023AC20FE03A780FF6F0080001307010065
:102B5000B7B300AA9B8303A0631C773A930180005C
:102B6000971000009380C04B3711A00A1B0101AAE7
:102B7000970700009387470123AE20FE03A7C0FFFD
:102B80006F00800013070100B713A00A9B8303AAFC
:102B900063107738930190009710000093804048AD
:102BA00037A10AA01B01A1009707000093874701E6
:102BB00023A0200003A700006F008000130701007E
:102BC000B7A30AA09B83A300631477349301A000EA
:102BD0009710000093800045375134121B01816724
:102BE000138200FE2320220283A20000B753341276
:102BF0009B838367639E72309301B000971000003F
:102C000093804042373121581B0181099380D0FFC6
:102C1000A3A3200017120000130202418322020026
:102C2000B73321589B8383096394722E9301C000AC
:102C300013020000B7D0BBAA9B80D0CD17110000B3
:102C40001301413C2320110003270100B7D3BBAA85
:102C50009B83D3CD631E772A1302120093022000B8
:102C6000E31A52FC9301D00013020000B7C0ABDAA4
:102C70009B80D0CC171100001301C1381300000055
:102C80002322110003274100B7C3ABDA9B83D3CCC7
:102C9000631077281302120093022000E31852FCFD
:102CA0009301E00013020000B7C0AADD9B80C0BC06
:102CB000171100001301013513000000130000007C
:102CC0002324110003278100B7C3AADD9B83C3BC63
:102CD000631077241302120093022000E31652FCC3
:102CE0009301F00013020000B7B0DACD9B80C0BBA7
:102CF00013000000171100001301C130232611003A
:102D00000327C100B7B3DACD9B83C3BB631277201F
:102D10001302120093022000E31852FC93010001F9
:102D200013020000B7B0DDCC9B80B0AB13000000F5
:102D3000171100001301012D1300000023281100BA
:102D400003270101B7B3DDCC9B83B3AB6312771CC0
:102D50001302120093022000E31652FC93011001AB
:102D600013020000B7E0CDBC9B80B0AA13000000A6
:102D700013000000171100001301C128232A1100BD
:102D800003274101B7E3CDBC9B83B3AA6312771835
:102D90001302120093022000E31652FC930120015B
:102DA00013020000171100001301C125B720110004
:102DB0009B8030232320110003270100B72311003B
:102DC0009B833323631677141302120093022000AF
:102DD000E31A52FC930130011302000017110000A6
:102DE00013014122B71001309B80302213000000F4
:102DF0002322110003274100B71301309B833322A4
:102E0000631877101302120093022000E31852FC9B
:102E10009301400113020000171100001301811EED
:102E2000B71000339B802012130000001300000035
:102E30002324110003278100B71300339B8323123F
:102E40006318770C1302120093022000E31652FC61
:102E50009301500113020000171100001301811AA1
:102E600013000000B70030239B802011232611009F
:102E70000327C100B70330239B832311631A77080C
:102E80001302120093022000E31852FC9301600128
:102E900013020000171100001301C11613000000F7
:102EA000B70033229B80100113000000232811007B
:102EB00003270101B70333229B831301631A7704AD
:102EC0001302120093022000E31652FC93017001DA
:102ED00013020000171100001301C11213000000BB
:102EE00013000000B73023129B801000232A11002A
:102EF00003274101B73323129B831300631A770022
:102F00001302120093022000E31652FC631A3000F1
:102F10001395110063000500136515007300000090
:0C2F20001305100073000000731000C0C7
:082F3000010101010101010191
:102F3800417373657274696F6E206661696C65644C
:102F48003A2061646472203E3D202831554C203C73
:102F58003C203132292026262061646472203C20DE
:102F68003633202A202831554C203C3C2031322948
:102F78000A00000000000000417373657274696FF5
:102F88006E206661696C65643A20212870745B3331
:102F98005D5B616464722F2831554C203C3C2031C4
:102FA80032295D2026203078303830292026262006
:102FB8006361757365203D3D203078660A00000026
:102FC800417373657274696F6E206661696C6564BC
:102FD8003A206E6F64650A00417373657274696F95
:102FE8006E206661696C65643A20757365725F6D01
:102FF800617070696E675B616464722F2831554C2B
:10300800203C3C203132295D2E61646472203D3DB4
:1030180020300A0000000000417373657274696F04
:103028006E206661696C65643A202122696C6C6562
:1030380067616C20696E737472756374696F6E2250
:103048000A00000000000000417373657274696F24
:103058006E206661696C65643A2070745B335D5BF1
:10306800616464722F2831554C203C3C2031322950
:103078005D20262030783034300A0000000000003F
:10308800417373657274696F6E206661696C6564FB
:103098003A2070745B335D5B616464722F2831552C
:1030A8004C203C3C203132295D20262030783038B5
:1030B800300A000000000000417373657274696F84
:1030C8006E206661696C65643A2074662D3E657091
:1030D8006320252034203D3D20300A0000000000F8
:1030E800417373657274696F6E206661696C65649B
:1030F8003A202122756E6578706563746564206571
:103108007863657074696F6E220A00000000000021
:10311800417373657274696F6E206661696C65646A
:103128003A202122756E737570706F727465642011
:0C31380073617470206D6F6465220A00E2
:10400000EFBEADDEEFBEADDEEFBEADDEEFBEADDED0
:10401000EFBEADDEEFBEADDEEFBEADDEEFBEADDEC0
:08402000EFBEADDEEFBEADDE28
:040000058000000077
:00000001FF
